:100000000C94A3020C94C0020C94C0020C94C00285
:100010000C94C0020C94C0020C94C0020C94C00258
:100020000C94C0020C94C0020C94C6270C94822736
:100030000C94C4280C94C0020C94C0020C94C0020E
:100040000C94C0020C94C0020C94C0020C94C00228
:100050000C94C0020C94A0280C94C0020C94C00212
:100060000C94C0020C94C0020C94C0020C94C00208
:100070000C94C0020C94C0020C94C0020C94C002F8
:100080000C94C0020C94C0020C94C0020C94C002E8
:100090000C94C0020C94C0020C94C0020C94C002D8
:1000A0000C94C0020C94C0020C94C002050109809B
:1000B000A101850319012AB700150126B700950192
:1000C00075108100C0050C0901A101850419012AE0
:1000D000A002150126A002950175108100C00660DE
:1000E000FF0961A1010962150026FF00952075082E
:1000F00081020963150026FF00952075089102C052
:1001000005010906A101050719E029E715002501E8
:10011000950875018102950175088101050719008F
:1001200029FF150026FF00950675088100050819AE
:10013000012905950575019102950175039101C08D
:10014000FD377A585A000004E6D6B4460200210171
:1001500016000000742FE5A3E002E7014F5D003DAB
:100160008889C65436C3174FE4E4678720B2EF3955
:100170006CB85B48EDEFAF45C7D8E1A4E6FAA147FC
:10018000C9CB33E3FE8991D3F9B5F3B849712E1386
:10019000AA90AB22B902099251EEF0F4E016797EF2
:1001A0004E116627E4762A31C02ADEBA0DCD891BAE
:1001B000ED770000733C2A2E1E85B3D4BD00884F16
:1001C000E32AE527F8B37F55950A320620E207486F
:1001D00044B986DB94849E90949089427118A3DA86
:1001E000324867B2E6ED8ECA19BEFA508B834B5C7B
:1001F0003234D255D1C638BC06D995802BE21A715B
:100200004CE4B7B58EFF508BDD034C86AFF7C5C904
:100210005FDFF957DAE0EAEE9A8CA349EB1F38600A
:10022000B41F6732D629D2901FBB0D2F10459D2CCD
:10023000145C58ADBC2CDA83AF194E6A8EDA1110FB
:10024000B7E57AAEBEA21091443EEA27A33EC9CAE2
:1002500049726AC1679DCAA0E59AC09069E4880E98
:10026000D4798FBAAC6509EEA96BF8D36E49EA0967
:1002700025E57018CDA876287CF9E6D419C3EDD60B
:10028000445C32B53CF22F6682381283177013E358
:100290002B24D85D654F0215B1EEB0335685EE853F
:1002A000656B509E0CC3B927551DFB9268DC00009E
:1002B000E7E341317AFC27500001EB02E80500003A
:1002C000C0C716D0B1C467FB020000000004595A31
:1002D000680069006A006B00AC00AE00AB00A800CB
:1002E000A900AA00000000000000000000000000BB
:1002F00001000100010001000100010001000100F6
:1003000001000100000000000000000000000000EB
:1003100001000100010001000100010001000100D5
:1003200001000100000000000000000000000000CB
:1003300001000100A503E40A160B00000200020000
:10034000A103E40A160B000003000100A603E40A5F
:10035000160B0000040002008B03E40A160BF105E3
:1003600005000100A703E40A160B000006000200C6
:100370008D03E40A160B000007000200A303E40A41
:10038000160B000008000100A803E40A160B000089
:1003900012000200A903E40A160B00001300020079
:1003A000AB03E40A160B000014000100AD03E40ADD
:1003B000160B000015000000000077057211000008
:1003C00009025B00030100A0FA0904000001030117
:1003D00001000921110100012240000705810308E5
:1003E00000010904010002030000000921110100BD
:1003F00001222200070582032000010705030320D4
:10040000000109040200010300000009211101009C
:1004100001223200070584032000011201000200BE
:1004200000000849501B000100010203011C037673
:1004300000690061006C003A006600360034006319
:1004400000320062003300630000002A035000699C
:10045000006B00610074006500610020004D0061C8
:1004600000630072006F00700061006400200047AC
:100470000042003400000018034A00610063006B72
:10048000005F004B0065007300740065007200009F
:100490000004030904000000000000000000000048
:1004A000000000000000000000000000000000004C
:1004B0000000000000000000007E0F00D4FFFFFFDE
:1004C000C70000007800000000000000002A2B2870
:1004D000000000000000000000000000000000001C
:1004E00029000000002C1E34202122243426272538
:1004F0002E362D3738271E1F202122232425263370
:1005000033362E37381F0405060708090A0B0C0D71
:100510000E0F101112131415161718191A1B1C1D83
:100520002F3130232D350405060708090A0B0C0D61
:100530000E0F101112131415161718191A1B1C1D63
:100540002F3130354C0011241FBECFEFDAE0DEBF73
:10055000CDBF11E0A0E0B1E0E6E6F0E602C0059014
:100560000D92AA37B107D9F724E0AAE7B1E001C09C
:100570001D92A939B207E1F70E94E7280C940630D2
:100580000C940000E8EDF0E080818E7F8083109273
:10059000E2001092DA001092E100A0EEB0E08C913F
:1005A00081608C9380818F77808319BCA7EDB0E048
:1005B0008C918E7F8C9380818F7E808310928004BB
:1005C00008952091E4003091E50095E6A90120917D
:1005D000EC00822F817020FF06C08091E80080FF30
:1005E00006C080E008952091E80022FD1AC08091A5
:1005F0008D04882389F0853089F08091EB0085FD9A
:100600000FC02091E4003091E50042175307F9F242
:100610009150E1F684E0089582E0089583E0089522
:1006200081E00895EF92FF920F931F93CF937C0187
:100630008B010E94E102C82F811117C08091E80050
:1006400085FD0BC08091E8008E778093E8000E94C2
:10065000E102882399F3C82F08C0F70181917F0137
:100660008093F1000150110949F78C2FCF911F9110
:100670000F91FF90EF90089580918F0487FF13C032
:100680008091E80082FF06C08091E8008B7780931C
:10069000E80004C080918D048111F2CF089580910B
:1006A0008D048823D9F38091E80080FFF8CF8091F2
:1006B000E8008E77ECCF982F9093E900242F762FC7
:1006C00050E0891731F07091EC002091ED005091CD
:1006D000F00021FD07C09F5F973071F78093E9001C
:1006E00081E008953091EB003E7F3093EB00309134
:1006F000ED003D7F3093ED003091EB0031603093A1
:10070000EB007093EC002093ED005093F0002091EB
:10071000EE0027FDE0CF80E00895B0E0A0E0E3E93F
:10072000F3E00C94452FC8EDD0E088818F7E88835C
:10073000E7EDF0E080818160808384E082BF81E02A
:100740008093800488818E7F888302EE10E0F80118
:1007500010821092DA0081EEC82ED12CF6011082A0
:1007600088818F77888388818068888388818F7D5E
:10077000888319BC10928D0410928E0410928C0400
:1007800010928B0490EEE92EF12CF70180818B7F83
:10079000808388818160888342E060E080E00E94FD
:1007A0005B03F60180818E7F8083F8018081816008
:1007B0008083808188608083F70180818E7F808341
:1007C000888180618883CDB7DEB7E8E00C94612F23
:1007D000FC01809195049091960486179707A0F0EC
:1007E0006115710529F49091E8009E779093E800D7
:1007F00090E06115710551F4911108C08091E800F5
:1008000082FF34C080E00895BC01F2CF80918D0456
:100810008823C1F18530C1F18091E80083FD30C0AB
:100820008091E80082FDEACF8091E80080FFE1CF6F
:100830008091F3002091F200382F6115710519F0B5
:100840002830310558F091E02830310509F090E06A
:100850002091E8002E772093E800CBCF8191809300
:10086000F100615071092F5F3F4FE7CF80918D04F8
:10087000882341F0853041F08091E80083FFBECFAE
:1008800081E0089582E0089583E008950895089531
:1008900080918204089587E797E7909301088093F9
:1008A000000888E19AE00FB6F894A895809360005C
:1008B0000FBE90936000FFCF9C014FB7F8948091DA
:1008C000790490917A04A0917B04B0917C044FBF8D
:1008D000821B930B08952FB7F8946091790470915F
:1008E0007A0480917B0490917C042FBF08952FB7E8
:1008F000F8948091790490917A04A0917B04B0914E
:100900007C042FBF08952091770430917804281734
:10091000390771F09093780480937704E09175041F
:10092000F0917604309721F00084F185E02D09954F
:10093000089520917304309174042817390771F0D9
:100940009093740480937304E0917504F09176049D
:10095000309721F00680F781E02D09950895E09108
:100960007504F0917604309729F00190F081E02D24
:100970000995089580E00895CF93DF93EC014091AD
:1009800063045091640460916504709166042FB70C
:10099000F8948091790490917A04A0917B04B091AD
:1009A0007C042FBF841B950BA60BB70B843F914093
:1009B000A105B10518F58091630490916404A0919C
:1009C0006504B091660480935F0490936004A093E3
:1009D0006104B093620484EF91E0A0E0B0E0809302
:1009E0005B0490935C04A0935D04B0935E04D09389
:1009F0006B04C0936A04DF91CF9108950E946B0449
:100A000060935F0470936004809361049093620428
:100A100082E390E0A0E0B0E0E2CFFC018481862395
:100A200051F492819923B9F06923808583FF05C031
:100A300081E061110FC080E00895892F8F70929539
:100A40009F70982B862F8F7062956F70682B81E056
:100A50009613F1CF089581E0FDCF452B39F068233F
:100A600081E06F3F09F080E08170089581E0FCCF64
:100A7000DC016091570480915804962F891301C0BE
:100A80000895292F30E0F901EE0FFF1FE15BFB4FC6
:100A9000408151814A175B07A1F487E08A9FA0013A
:100AA0008B9F500D1124495E5B4F81E0FA018483D6
:100AB0009613E6CF2F5F3F4F2370332720935704C1
:100AC00008952F5F3F4F922F9370D8CF1092B403A9
:100AD0001092B303E7E1F4E08581811102C0148232
:100AE0001682379684E0EF34F807B1F70895B0E046
:100AF000A0E0EDE7F5E00C94432F8FEF9FEF44303B
:100B0000510508F469C04091680341FB882780F9CA
:100B100090E0880F991F42FB002700F910E0000FBA
:100B2000111F000F111F802B912B40FBCC24C0F80C
:100B3000D12C8C299D2943FB222720F9C22FE0E0EC
:100B4000DE2F53E0CC0FDD1F5A95E1F78C2B9D2B48
:100B500044FBAA27A0F9B0E0E4E0AA0FBB1FEA9586
:100B6000E1F78A2B9B2B45FBEE27E0F9F0E0A5E0AF
:100B7000EE0FFF1FAA95E1F78E2B9F2B46FB222736
:100B800020F930E0B6E0220F331FBA95E1F7822B4F
:100B9000932B47FB222720F930E03695322F22276E
:100BA00037952795822B932B20916903322F317033
:100BB000F32EE82EF92A26952170B22EBB0CA82E12
:100BC000BF28C501BB0CAA0BBB0BFB018083918323
:100BD000A283B38390E080E0CDB7DEB7EAE00C9467
:100BE0005F2F80918B0390918C03909310018093E1
:100BF0000F010895E9E1F2E090E080E061E276E241
:100C000048E456E226E935E27783668351874087D8
:100C1000338722879587848701963E968830910591
:100C200099F7089581152CE5920741F420910D0163
:100C300030910E01232B11F490E080E0089580E0C4
:100C40000895F894E82FE295EF70F0E031A1282F95
:100C50002F7081E090E001C0880F2A95EAF7982F65
:100C60009095932391A392A1892B82A378940895C0
:100C70009091680392FF06C0282F28712830F9F45C
:100C8000877F846093FF06C0282F28712831F1F4F4
:100C9000877E84612091690320FF06C0382F387158
:100CA0003830D9F4877F816021FF06C0282F287152
:100CB0002831D1F4877E816194FD877E0895282FA5
:100CC00024712430F9F68B7F8860DCCF282F2471C3
:100CD000243101F78B7E8861DDCF382F31713130BF
:100CE00019F78E7F8860E0CF282F2171213121F7FD
:100CF0008E7E8861E1CFCF93DF93EC01823891053E
:100D0000B1F108F040C08133910509F49DC048F568
:100D10008932910509F48DC08A9709F49CC0C115E8
:100D200022E5D20708F0BDC0C11531E5D30708F0B0
:100D300025C1C83ED10508F0A3C0C13ED10588F544
:100D4000C83AD10508F08EC0C53AD10508F0F6C002
:100D5000C130D10531F1209721F1C430D10508F51A
:100D600045C08533910509F45FC0C997C1F68091EC
:100D70006803837009F037C18091690383FF11C054
:100D8000C9E2D0E00EC0833E910599F170F4803E37
:100D9000910501F1823E910511F68091680382FD73
:100DA00021C0CE01DF91CF910895863E910561F17A
:100DB000873E910571F1843E910509F0B0CF809195
:100DC000690381FFEECF80916803C7EED0E084FD18
:100DD0000DC0E7CF8091680380FD33C09091690317
:100DE00090FFDFCFC3EED0E084FFDBCFD0E0C0E0E8
:100DF000D8CF8091680382FDF3C09091690390FD84
:100E0000F2C084FFCECFF2CF8091680383FDDDCFA7
:100E1000C8CF8091680383FDE9C09091690391FF79
:100E2000F0CFC4EED0E0BDCF8091680385FFB9CF8D
:100E3000A7CF8091680385FDDCC08091690383FFA3
:100E4000B0CFC9E3D0E0ADCF8091680386FFA9CFD2
:100E5000CAE2D0E0A6CF8091680386FFA2CFC1E3AB
:100E6000D0E09FCFCF3BD10508F6C85AD0E0CC0FD9
:100E7000DD1FC15EDE4F0990D881C02DD46491CFB3
:100E8000C11540E5D40708F064C0C11580E4D80757
:100E900008F05CC0CE019A9581159F4108F481CF7E
:100EA000A5CFC11536E5D30718F5C11545E5D4071B
:100EB00008F07DC0C11584E5D80708F073C09C2FE9
:100EC000969596959E0123703327C115D34508F456
:100ED0005AC0C1E0D0E002C0CC0FDD1F2A95E2F776
:100EE00030E2939FC0011124C82BD92BDA6859CF67
:100EF000C1158AE5D80778F4C11529E5D20708F0AD
:100F000061C0C11538E5D30708F470CFDC2FCC27BA
:100F1000C06FD06A46CFCE0190568115904208F03E
:100F200065CF8D2F8F710E94380690E0982F88270B
:100F300088279F719C012C2BE90142C0C55AD0E043
:100F4000C45EDE4FC881D0E0D0642BCFDF70D06AA2
:100F500028CF2C2F26952695237080E2289F90017C
:100F600011248C2F8370C1E0D0E002C0CC0FDD1FB4
:100F70008A95E2F7C22BD32BDD6813CFDC2FCC2769
:100F8000C16FD06A0ECFC1E0D0E002C0CC0FDD1F30
:100F90002A95E2F720E2929FC0011124C82BD92B99
:100FA000DC68FFCEDC2FCC27C46FD06AFACE8C2F42
:100FB0000E943806C82FD0E0DC2FCC27CC27DF7169
:100FC000D062EFCE8C2F8F700E94380634E0D69519
:100FD000C7953A95E1F7CF709C2FEC01D069E1CE2F
:100FE000C2EED0E0DECEC0EED0E0DBCEC6EED0E08A
:100FF000D8CEC5E3D0E0D5CE8091E701882331F08B
:101000001092E7011092E6011092E5010895CF9346
:10101000C82F8091690382FF0CC08091E7018C1773
:1010200041F00E9477049093E6018093E501C0931C
:10103000E701CF910895809590919804982390931B
:1010400098040895809590916A03982390936A0379
:10105000089590916A03892B80936A0308951092F2
:10106000DC011092DB011092DA01089580918D036A
:1010700090918E03892B89F00E9477042091E501DD
:101080003091E601AC01421B530B81E020918D03AE
:1010900030918E034217530708F480E08170089561
:1010A000EEE7F1E09191891303C0DF0111971C92E3
:1010B00091E0E438F907B1F70895AEE7B1E0EFEF5A
:1010C00090E02D91821751F0EF3F19F4211101C0EA
:1010D000E92F9F5F9630A9F7EF3F09F408950E2E90
:1010E000000CFF0BE458FE4F828308952091D90134
:1010F00090919801291302C080E0089530E0F90131
:1011000053E0EE0FFF1F5A95E1F7E756FE4F51816E
:10111000561306C05081581303C05281541304C0A3
:101120002F5F3F4F2770E6CF81E008958091D9016E
:1011300090919801981301C008958F5F8770FACF3E
:10114000923080F5883070F548E0949F900111242A
:10115000820F932F911D682F677023E096958795D6
:101160002A95E1F7FC01EE0FFF1FE80FF91FE65784
:10117000FE4F50E040E080E0219130E0062E02C0BA
:10118000369527950A94E2F721703327042E01C083
:10119000220F0A94EAF7822B4F5F5F4F43305105CD
:1011A00059F7089580E00895923098F5883088F5D1
:1011B00048E0949F90011124820F932F911D282FB6
:1011C000277041E001C0440F2A95EAF723E0969585
:1011D00087952A95E1F7FC01EE0FFF1FE80FF91F35
:1011E000E657FE4F90E080E070E05191DF011197EB
:1011F0009B01082E02C0369527950A94E2F72170CC
:1012000021952527242325272C93019683309105AA
:1012100061F7089592959F70963091F058F4925F1F
:101220009F70923058F4803F19F030F4883E30F4CB
:1012300081E008959A5FF4CF843FD1F380E0089570
:10124000883EB0F3813FD1F7F3CF9C013A95211549
:101250003F4150F5FC01EE27F170BC01662772702A
:10126000AC01442754709C012227387094FF0EC0B3
:1012700080E1EF2B09F480E0672B09F08062452BB9
:1012800009F08064232B89F08068089581E0EF2BBA
:1012900009F480E0672B09F08260452B09F0846037
:1012A000232B19F08860089580E0089580937D04D1
:1012B00070937F0460937E0480918D048430F9F4F0
:1012C0008093E9008FEF9091E800815095FD06C072
:1012D0009AE69A95F1F700C08111F5CF8091E80068
:1012E00085FF0DC050E040E063E070E08DE794E0E2
:1012F0000E9412038091E8008E778093E8000895A1
:10130000BC0184E00E9456090895BC0183E00E945C
:1013100056090895CF93DF93EC0181E08093E900B3
:101320008FEF9091E800815095FD06C09AE69A955E
:10133000F1F700C08111F5CF8091E80085FF14C05E
:1013400050E040E068E070E0CE010E94120380911E
:10135000E8008E778093E80088E0FE01A3E8B4E01F
:1013600001900D928A95E1F7DF91CF910895019751
:1013700008F40895EFECF7E03197F1F700C00000B2
:10138000F6CF0F931F93CF93DF930BE813E0C3E9DE
:10139000D0E0CE010E94BC2FF80181938F012196ED
:1013A000C73BD105B1F7CAE3D3E0FE018591949123
:1013B000009711F0FC0109952C96F3E0CA3CDF0779
:1013C000A1F7DF91CF911F910F9108950F931F9374
:1013D000CF93DF93833038F5623028F5483018F525
:1013E00020E1629F8001112450E0440F551F040F3B
:1013F000151F30E2839FC0011124080F191FC80177
:1014000087960E94BC2FC82FD0E0DC2FCC27C801C4
:1014100088960E94BC2F9E01282BC901DF91CF9195
:101420001F910F91089590E080E0F8CF462F209112
:10143000660330916703232B99F4703F39F4603FC2
:1014400079F480916403909165030895833040F4AA
:10145000723030F4683020F4672F0E94E609089556
:1014600090E080E00895CF92DF92FF920F931F9358
:10147000CF93DF936C01009197048091E801082BD2
:10148000C7E0D0E010E0FC2EC8010C2E02C09595FC
:1014900087950A94E2F780FD0CC02197A0F7F12C04
:1014A0008F2DDF91CF911F910F91FF90DF90CF9003
:1014B0000895B6018C2F0E94160A0E947B060197A0
:1014C00061F3EECFCF93DF93EC010E94330ABE01AC
:1014D0000E94160A0E947B06DF91CF910895CF9358
:1014E000DF93EC014B815C81698188810E942D052D
:1014F000811110C08E819F81009739F00E947B0678
:101500000E940A09DF91CF910895888199810E94F4
:10151000620AF6CF80E0F6CFA5E0B0E0E2E9FAE0BB
:101520000C944A2F49835A8389819A81662399F0C2
:10153000222389F00E94330A182F682F89819A810B
:101540000E94D40869817A81812F0E94160A25960B
:10155000E3E00C94662F0E94A008182FF3CFFC0143
:10156000262F86819781009739F4408151816281CD
:10157000738184810E948C0A089583E290E00E9426
:10158000BC2F8E3D89F484E290E00E94BC2F833C06
:1015900059F485E290E00E94BC2F91E08A3009F076
:1015A00090E0892F8170089580E0FCCFCF9384E094
:1015B00090E00E94BC2FC82F82E290E00E94BC2FD6
:1015C000982F8C2FCF910895DB01FC013296259145
:1015D00034914217530758F0FC0134966591749189
:1015E000A901CD010E949C2F90E080E008958FEF2B
:1015F0009FEF08950F931F93CF93DF930BE813E0B2
:10160000C3E9D0E0CE010E94BC2FF80161918F01A7
:10161000681719F0CE010E94CA2F2196C73BD10549
:1016200089F7DF91CF911F910F910895DA019C0105
:101630002E5F3F4FF90145915491F9012591349165
:10164000A217B30758F0FC013496859194910E943B
:101650009C2F0E94FA0A90E080E008958FEF9FEFA0
:101660000895CF93DF93C7EAD1E060E0CE010E94F6
:10167000CA2F2196C11584E0D807B9F7DF91CF9121
:1016800008951F93CF93DF93122F8330E8F46230D5
:10169000D8F44830C8F420E1629FE001112450E002
:1016A000440F551FC40FD51F20E2829FC001112493
:1016B000C80FD91F632FCE0187960E94CA2F612FB2
:1016C000CE0188960E94CA2FDF91CF911F91089575
:1016D000CF93C82F6FEF81116EED83E290E00E94EF
:1016E000CA2F6FEFC11163EC84E290E00E94CA2F11
:1016F0006FEFC1116AE085E290E00E94CA2FCF919E
:101700000895CF93C92F682F84E090E00E94CA2FDC
:101710006C2F82E290E00E94CA2FCF9108959B0126
:10172000883070F49AE0899FB001112469547F4F8A
:101730004AE050E0C9010E94AC2F90E080E008959B
:101740008FEF9FEF0895AAE0B0E0E9EAFBE00C9488
:101750004B2F9C0137552F3F310509F068F4BE012E
:101760006F5F7F4F0E948F0B892B31F489859A859B
:101770002A96E2E00C94672F8091A3039091A40332
:10178000F7CFAAE0B0E0E7ECFBE00C94412F0CEEC1
:1017900012E08AEDC82E82E0D82E97E5E92EFF24CC
:1017A000F39427E0922E39EDA32E32E0B32E882455
:1017B0008394D6010D931D936D014AE050E0B7016B
:1017C000CE0101960E94AC2FF8013896DF01892DD9
:1017D0001D928A95E9F789819A81D80111969C9387
:1017E0008E938F8112968C9312978D8113968C9382
:1017F0001397888514968C931497898515968C93E6
:1018000015978B819C8117969C938E9316971896AB
:101810001C9218978A8587FF3CC01E961C921E92C8
:101820001D9780FF03C0D80118968C9281FF04C0D9
:10183000F80190859260908782FF07C0D8011896C2
:101840009C911897946018969C9383FF04C0F801AC
:1018500090859860908784FF07C0D80118969C9166
:101860001897906118969C9385FF04C0F8018085B5
:1018700080628087015F1F4FFAE0EF0EF11C87EA5C
:10188000E81681E0F80609F094CF2A96ECE00C9473
:101890005D2FF801B686A586C4CFAAE0B0E0E3E5E7
:1018A000FCE00C94452FE9E8F2E080E5DF011D92B1
:1018B0008A95E9F7E7E1F4E088E3DF011D928A9574
:1018C000E9F789E8C82E82E0D82E7F0107E011E011
:1018D000F701D182C0824AE050E0B801CE01019602
:1018E0000E94AC2F88E0FE013196D60101900D9246
:1018F0008A95E1F789859A85D70113969C938E93F3
:101900001297BAE0CB0ED11CE7E0EE0EF11C065F99
:101910001F4F0735F1E01F07D9F62A96E8E00C942F
:10192000612F80916A0390919804892B80937C01A8
:101930008091E701882309F180918D0390918E03B6
:10194000892B29F00E94360881110E94FC078091A2
:101950007C019091E701892B80937C0120E08EE748
:1019600091E0FC013191CF0131112F5FF1E084381A
:101970009F07B9F721110E94FC07809167048095A9
:1019800090917C01892390916804892B80937C013C
:1019900048E050E06DED71E08CE791E00E948F2F00
:1019A000892BA9F088E0ECE7F1E0ADEDB1E0019022
:1019B0000D928A95E1F7E0917504F09176043097E5
:1019C00031F00280F381E02D8CE791E009950895D4
:1019D000CF93DF93EC01EA85FB85309719F06C8596
:1019E0007D8509958B810E941B088C810E942208AD
:1019F0000E94910C86E0FE0111928A95E9F7DF9131
:101A0000CF910895CF93DF93EC018D8181FD15C0B7
:101A100082608D83809198049B81892B80939804A8
:101A20008C810E9429080E94910CE885F9853097E5
:101A300021F06C857D85CE0109951092720410927B
:101A400071048D8180FD03C0CE010E94E80CDF91FE
:101A5000CF91089580911101877F8093110182E0D9
:101A60000E941B088091110184FF06C08F7E809325
:101A7000110182E00E9429088091110185FF06C0B2
:101A80008F7D8093110180E20E9429080E94910CB1
:101A9000089590E080E00E94990490E080E00E9428
:101AA0008304109298040E94910C089580939704E7
:101AB0000E94490D089580919704982F9670963052
:101AC00021F488600E94560D0895877FFBCF21E0A6
:101AD00030E001C0220F8A95EAF7209580919704A3
:101AE00082230E94560D08959091DC0180958923F0
:101AF0008093DC01282F277091F4282F082E000CEA
:101B0000330B9217130659F09091690392FF07C0A7
:101B10008595859585950E94670D0E942F080895EB
:101B20009091690392FB222720F9281769F080FB26
:101B300092F99093690380916803909169030E94E0
:101B4000810B82E00E94740D089521E030E001C015
:101B5000220F8A95EAF780919704822B0E94560DF6
:101B600008959091690392FF10C098E0899F9001B9
:101B70001124622B6093DC010E94A50D0E94770462
:101B80009093DB018093DA0108950E94A50D0895DA
:101B90008093E8010E94490D089510926A03EEE7D0
:101BA000F1E086E0DF011D928A95E9F70E94490D78
:101BB0000895AAE2B0E0EFEDFDE00C944A2F8FE823
:101BC00094E02091F100DC012D93CD01B4E0873940
:101BD0009B07B9F780919004833009F472C0B8F480
:101BE000813009F449C0823009F4B3C08091E80023
:101BF00083FF96C280918F04909190049A3008F0F0
:101C00008FC2E92FF0E0E85FFF4C0C942E2F8A3052
:101C100009F48EC08B3009F471C0893039F7809196
:101C20008F04813219F78091930490919404009766
:101C300011F00297D9F68091E800877F8093E80041
:101C40008091E80082FF38C09091F3008091F2000B
:101C5000029731F48091F100813011F0863021F447
:101C60008091F100809382048091E8008B778093CB
:101C7000E8000E943C03BACF80918F04813A09F0BA
:101C8000B5CF8091E800877F8093E800809193042E
:101C900090919404892B61F468E083E894E070E00B
:101CA0000E94E8038091E8008B778093E8009ECF44
:101CB00060E090E080E0F3CF80918D048111C0CF8F
:101CC00095CF80918F04813A09F090CF8091930451
:101CD00090919404892B09F089CF8091E800877F47
:101CE0008093E8008091E80080FFFCCF8091130191
:101CF0008093F1008091E8008E77B9CF80918F04B6
:101D0000813209F073CF8091930490919404892BD0
:101D100009F06CCF8091E800877F8093E8000E94F3
:101D20003C0380919104809313010E94CD0D5ECFFE
:101D300080918F04813209F059CF8091E800877F2C
:101D40008093E8000E943C03809192048093810478
:101D50004DCF80918F04813A09F048CF8091E800FF
:101D6000877F8093E8008091E80080FFFCCF80911E
:101D70008104BECF803899F0823809F0D1C18091BA
:101D800093048F70873008F0CBC18093E900809175
:101D9000EB0085FB882780F91092E90006C080914E
:101DA0008B0490918C04911182609091E800977F50
:101DB0009093E8008093F1001092F1008091E80088
:101DC0008E77AAC1882309F498C1823009F0A8C18E
:101DD0008091910481119BC1809193048F702FEFAA
:101DE000280F263008F09CC18093E9002091EB0079
:101DF00020FF8DC1933031F48091EB00806280939D
:101E0000EB0085C19091EB0090619093EB0021E095
:101E100030E001C0220F8A95EAF72093EA00109281
:101E2000EA008091EB008860EACF811179C11091BE
:101E300091041F778091E3008078812B8093E300E9
:101E40008091E800877F8093E8000E943C038091A6
:101E5000E80080FFFCCF8091E30080688093E3007E
:101E600082E0111183E080938D045AC18058823042
:101E700008F056C120919104309192042C3DE3E08A
:101E80003E07A1F583E08A838AE289834FB7F894FD
:101E9000DE01139620E03EE051E2E32FF0E05093A4
:101EA0005700E49120FF03C0E295EF703F5FEF70B1
:101EB0008E2F90E0EA30C0F0C7968D939D932F5FF0
:101EC000243159F74FBF8091E800877F8093E80065
:101ED0006AE270E0CE0101960E94E8038091E8007A
:101EE0008B778093E8001CC1C096E7CF8091930464
:101EF00090919404432F55274330510509F44AC06B
:101F000078F54130510509F485C08BE590E0E0ECAF
:101F1000F3E04230510509F003C12091E800277F2A
:101F20002093E8002091950430919604821793073E
:101F300008F49C0140E02115310509F070C0411101
:101F40006EC08091E80082FDC9CF80918D04882306
:101F500029F2853019F28091E80083FFF2CFBECFDD
:101F60004132510509F447C04232510509F0D8C049
:101F70008330910508F0D4C0FC01EE0FFF1FE25939
:101F8000FE4F0190F081E02D85599E4FDC018C9130
:101F900090E01DC0332721303105E9F021153105CE
:101FA00079F022303105F9F02330310509F0B8C05D
:101FB000EDE2F4E0E4918E2F90E0EDE2F4E007C072
:101FC000E1E9F4E0E4918E2F90E0E1E9F4E000979C
:101FD00009F4A6C0A2CFE7E7F4E0E4918E2F90E0E9
:101FE000E7E7F4E0F4CFEBE4F4E0E4918E2F90E047
:101FF000EBE4F4E0ECCF8330910508F091C0880F5A
:10200000991FFC01EC58FE4F0190F081E02D89E012
:1020100090E083CF82E190E0EBE1F4E07ECF80912D
:102020008D04882309F45ACF853009F457CF809165
:10203000E80083FD53CF8091E80082FD82CF80913C
:10204000E80080FF78CF9091F3008091F200211595
:10205000310519F08830910550F041E0089709F0FA
:1020600040E08091E8008E778093E80064CF44914F
:102070004093F1003196215031090196E8CF803824
:1020800009F04EC08091E800877F8093E80080913E
:102090008E048093F10092CE811142C01091910480
:1020A0001230F0F58091E800877F8093E80010936C
:1020B0008E040E943C03112311F084E005C080913E
:1020C000E30087FDFACF81E080938D0442E061EC6C
:1020D00081E00E945B0342E261EC84E00E945B03CA
:1020E00042E261EC82E00E945B0342E260EC83E04A
:1020F0000E945B0380918D0413C080919104813014
:1021000079F481E0933009F080E080938C041092A0
:10211000E9008091E800877F8093E8000E943C03FB
:102120008091E80083FF0AC08091E800877F809358
:10213000E8008091EB0080628093EB00AA96E3E0D8
:102140000C94662FEBE8F3E0128E138E8FEA90E08A
:102150009183808385E0848F28E833E13383228371
:1021600022E330E0378B268B28EC30E0318F208F54
:10217000158E178E168E20E530E031A320A382A3A2
:102180000E94FA0A0E94CD0D109269031092680312
:10219000E9E6F3E080818460808380916803909118
:1021A00069030E94810B0E94C1090895AEE1B0E06D
:1021B000ECEDF0E10C94402FA0900D01B0900E01D9
:1021C00081E090E090930E0180930D0180EDC82E88
:1021D00082E0D82E10E07601712C16C0F401259112
:1021E0003491402F672D812F0E94410B82E0880E91
:1021F000911C0F5F083091F7E0E1EE0EF11CF1E069
:102200007F1629F077247394470100E0E7CF1F5F22
:1022100080E2C80ED11C1330F1F60E94A2101A827F
:1022200019821C821B821E821D8218861F8288ECE6
:1022300090E09A87898707EB10E04AE050E0B80108
:10224000CE0101960E94EE2F065F1F4F0730E1E09E
:102250001E0799F77E01FBE0EF0EF11C8AE0F70103
:1022600011928A95E9F74AE050E0B801C7010E944F
:10227000EE2F065F1F4F0735F1E01F07A1F77E0124
:1022800085E1E80EF11C8AE0F70111928A95E9F7E1
:102290008FEF9FEF9A8F898F87E08E8F4AE050E013
:1022A000B801C7010E94EE2F065F1F4F073AF1E009
:1022B0001F07A1F7B0920E01A0920D016E96EDE0FE
:1022C0000C945C2F80E00E94680B60E086E290E056
:1022D0000E94CA2F0E94D6100E94310B81E00E94FA
:1022E000680B0895CF92DF92EF92FF928FEF9FEFEE
:1022F0004430510508F46AC0FB01C080D180E280FF
:10230000F3800E94CD0D80916803C0FA80F9B70177
:10231000A601769567955795479540FB81F9B701DA
:10232000A60122E076956795579547952A95D1F7AE
:1023300040FB82F9B701A60133E076956795579582
:1023400047953A95D1F740FB83F9B701A601E4E040
:102350007695679557954795EA95D1F740FB84F9AF
:10236000B701A601F5E07695679557954795FA95DB
:10237000D1F740FB85F9B701A601A6E076956795F0
:1023800057954795AA95D1F740FB86F9B701A60165
:10239000B7E07695679557954795BA95D1F740FB85
:1023A00087F98093680380916903D0FA80F9D1FAA4
:1023B000CC24C0F8C0FA81F9809369038091680346
:1023C000909169030E94810B90E080E0FF90EF9074
:1023D000DF90CF9008950E94CD0D2FE78AE196E01F
:1023E000215080409040E1F700C0000088E19AE071
:1023F0000FB6F894A895809360000FBE909360008C
:10240000FFCF882321F00E941B080E94910C0895A1
:10241000882339F090919804982B909398040E9407
:10242000910C0895882321F00E9422080E94910CAB
:102430000895882321F00E9429080E94910C089594
:10244000882309F44DC0823879F40E94AF0481FFDB
:1024500047C089E30E945D080E94910C89E30E94B5
:1024600050080E94910C0895833859F40E94AF04DB
:1024700080FF36C083E50E945D080E94910C83E5D1
:10248000EECF843859F40E94AF0482FF29C087E45C
:102490000E945D080E94910C87E4E1CF9CEF980FA9
:1024A000913AE8F290E2980F983050F4877091E0FA
:1024B00001C0990F8A95EAF7892F0E942208D1CF8F
:1024C0009BE5980F933028F490E080E00E949904F7
:1024D0000895885A873120F490E080E00E948304B8
:1024E0000895FF920F931F93CF93DF93F82E0091DF
:1024F0006C0410916D040115110509F449C0109286
:102500006B0410926A041092670410926804D80158
:102510001696CD91DC919E013A9521153F4108F424
:10252000D07ED1E0C11101C0D0E0D8011996ED9163
:10253000FC911A97309731F01B966D917C9180E059
:102540000995D823DD2339F08CEF8C0F813A30F5D3
:102550008C2F0E945008FF2099F0E0916C04F091BC
:102560006D04808584FD0CC080916904882341F04E
:10257000808191819C0121503109203B3D45A0F093
:102580000E94910C10926D0410926C0410926904D8
:10259000C801CDB7DEB7E5E00C94642F0E94910C22
:1025A0008C2F0E942012D7CF0E94BC04E9CFCF937A
:1025B000DF93EC010E942012CE010E9425099E01AA
:1025C000205E31092830310510F0CD2B29F40E940E
:1025D0001212DF91CF9108950E940112FACFCF938A
:1025E000C82F8823C9F08238C9F40E94AF0481FD46
:1025F00013C089E30E945D080E94910C2FEF83EFC6
:1026000091E0215080409040E1F700C0000089E354
:102610000E9450080E94910CCF9108958338A1F434
:102620000E94AF0480FDF8CF83E50E945D080E9400
:10263000910C2FEF80E792E0215080409040E1F72D
:1026400000C0000083E5E4CF8438A1F40E94AF0409
:1026500082FDE2CF87E40E945D080E94910C2FEF7B
:1026600080E792E0215080409040E1F700C00000F8
:1026700087E4CECF8CEF8C0F813A68F4EEE7F1E07F
:102680008191C81781F121E0E438F207C9F78C2F56
:102690000E945D08BFCF80E28C0F883048F4C7707D
:1026A00081E001C0880FCA95EAF70E942908B2CFDD
:1026B000EBE5EC0FE33040F4F0E0E45EFE4F8081A8
:1026C00090E00E949904A8CFC85AC73108F0A4CF5F
:1026D000EC2FF0E0EE0FFF1FE15EFE4F8081918155
:1026E0000E94830499CF8C2F0E9450080E94910C65
:1026F000CECF1F93CF93DF93182FC091AB03D09110
:10270000AC03893321F0C091A903D091AA03812F92
:102710000E94EF12209739F4812F0E942012DF913E
:10272000CF911F9108958FEC97E00197F1F700C0CA
:1027300000002197EFCFB0E0A0E0E1EAF3E10C94D4
:10274000432FEC018AE0A82E2881222309F48FC0B0
:102750002130C9F599818A81913021F422960E9415
:10276000791305C0923029F422960E94EF12219627
:10277000EBCF933021F422960E942012F8CF9430B0
:1027800011F02196F4CF229630E020E0AE014F5FA9
:102790005F4F8053990B8A30910550F021503109D9
:1027A00030F38FEC97E00197F1F700C00000F6CF0F
:1027B000A29EB001A39E700D11249C01260F371F0D
:1027C0008981EA01E3CFE22FF0E0EB53FB4FB490B5
:1027D000822F86958695869590E0FC01EB54FB4F01
:1027E000E4902770F12C022E02C0F594E7940A942D
:1027F000E2F731E0E322FF24FC01EB55FB4FC490EC
:10280000D12C022E02C0D594C7940A94E2F731E08D
:10281000C322DD24FC01EB56FB4F049110E002C003
:10282000159507952A95E2F701701127E114F10437
:1028300019F081EE0E94EF12C114D10419F086EE56
:102840000E94EF128B2D0E947913C114D10419F04C
:1028500086EE0E942012E114F10419F081EE0E942C
:1028600020120115110509F482CF8CE278CFCDB783
:10287000DEB7EAE00C945F2FB0E0A0E0E2E4F4E120
:102880000C94432F7C015B01C42FD22FFC01828169
:102890008823A9F0409370040E94770490936F04FA
:1028A00080936E04C77081E001C0880FCA95EAF773
:1028B0000E941912CDB7DEB7EAE00C945F2F109199
:1028C0007004141338C080916E0490916F040E94BC
:1028D0005C046C01B701C5010E94A30BC816D906A0
:1028E00050F5C0E2CD0F1D17C1F080E2810F883096
:1028F00048F4177081E0012E01C0880F0A94EAF7AE
:102900000E941212C83048F481E09D2F977001C0D8
:10291000880F9A95EAF70E941912802F0E94791366
:10292000C83040F6D77081E001C0880FDA95EAF729
:102930000E941212BFCFC77081E001C0880FCA95F4
:10294000EAF7F6CFCF93DF93EC010E9425099E01B1
:10295000205E31092830310510F0209741F40E94A3
:1029600019128C2F0E94EF12DF91CF9108950E94CF
:102970000812F7CF662329F0209198042260209353
:1029800098049C013056211540E2340720F0305E57
:102990002115304108F499270E94A2140895B0E04F
:1029A000A0E0E5EDF4E10C94462F7C018B01D42EE0
:1029B0008091110182FF8CC0C091B103D091B2030C
:1029C000CE15DF0521F0E114F10409F081C08091FA
:1029D00011018B7F8093110181FD73C08091AF0342
:1029E0009091B003A801481B590B81E020910F0181
:1029F000309110014217530708F480E08170F82EDF
:102A000080911101F0FA81F980931101FE0183E0B8
:102A1000F695E7958A95E1F7EE71FF27E559FC4FAA
:102A200020813181AE014F70552781E090E002C0D6
:102A3000880F991F4A95E2F7FF2009F444C0822BC2
:102A4000932B9183808380916A0381FF08C08091DA
:102A5000110180618093110182E00E94220880911F
:102A60006A0385FF08C08091110180628093110183
:102A700080E20E9422086F2DCE010E94BA14DD2050
:102A800031F08091A60385FF02C086FF3BC0809194
:102A9000A9039091AA030E94B7098091B103909174
:102AA000B2039C013056211540E2340720F0305E1D
:102AB0002115304108F499270E94D7120E942A0D4F
:102AC0001DC081E09BCF8095909582239323B9CF41
:102AD000C701992797013056211540E2340728F0A5
:102AE000305E2115304108F0C7010E94D712809155
:102AF000B1039091B2038E159F0501F31093B003BB
:102B00000093AF03CDB7DEB7E7E00C94622F68EE19
:102B10007EEF90E080E00E94E82F60E082E090E0AD
:102B20000E94CA2F60E083E090E00E94CA2F1092BA
:102B3000E80160E084E090E00E94CA2F64E082E255
:102B400090E00E94CA2F60E085E090E00E94CA2FCA
:102B500060E086E090E00E94CA2F6FEF87E090E08F
:102B60000E94CA2F40E050E0BA0188E090E00E9445
:102B7000DC2F60E08DE090E00E94CA2F40E050E042
:102B8000BA0188E190E00E94DC2F60E087E190E0EC
:102B90000E94CA2F40E050E0BA018CE190E00E9410
:102BA000DC2F70E060E080E290E00E94E82F40E0DF
:102BB00050E0BA0188E190E00E94DC2F80E00E94A2
:102BC000680B0E94621140E050E0BA018FE090E093
:102BD0000E94DC2F40E050E0BA0183E190E00E94C7
:102BE000DC2F0895A7E0B0E0E8EFF5E10C943B2F6F
:102BF0007C01DC0113964D915C91149711966C91B8
:102C000011978C910E942D058111EEC061E0C701E2
:102C10000E94AF0A8C01F70182818823E1F0809144
:102C20007104909172040097B1F00817190799F098
:102C3000FEE08F9FC0011124FC01E25EFD4F208168
:102C400024602083875E9D4FDC010D931C930E94BE
:102C5000020D10929804F7018281882311F40C94DC
:102C6000A41EC80182519F45409710F00C94981EF5
:102C70008FEF93E00E94BC2F8111A6C07EEED72E6D
:102C8000D00E07EA11E0D11036C019821A821B82D9
:102C90001C8299249A9468012FEFC21AD20AC801A3
:102CA0000E94BC2F89831A82882309F48DC0813049
:102CB00009F07FC0580132E0A30EB11CC6010E948A
:102CC000BC2FC82E8A83882309F47EC0C5010E94C8
:102CD000BC2FD82E8FEF8C0D8330D8F4580143E0F1
:102CE000A40EB11CDB82DD2021F0CE0101960E94F2
:102CF0009B138501D0CF0115F4E01F0709F464C0D0
:102D0000C8010E94BC2F811101C0DA940F5F1F4FD0
:102D1000BACF8BEF8C0D833030F5C8010396DB8280
:102D20005C01DD2031F3580154E0A50EB11C0E9476
:102D3000BC2F8C838823E9F28B819C818130AFEF9B
:102D40009A0710F0982F8827B6E0CB1631F0E7E00D
:102D5000CE1631F00E941026CCCF0E94EA25C9CFB2
:102D60000E947125C6CFF4E0CF12C3CF580124E0F2
:102D7000A20EB11CC80103960E94BC2FDD2021F1D8
:102D8000882311F18150990B989E9001999E300DE6
:102D900011244D2D4150550BCA01820F931F0197ED
:102DA00008F4A7CFAFECB7E01197F1F700C000002F
:102DB000F6CFCE0101960E949B1356019ACF81E077
:102DC0000E94A50D0E945B0D8091DC01877061F06F
:102DD000D70112968C91882339F08091690382FF84
:102DE00003C082E00E94740D2796E2E10C94572FF5
:102DF00081E00E94670DE6CF82E0FBCF823009F0D0
:102E0000E1C78091130290911402892B09F4DAC76B
:102E10002EE02C9DC0012D9D900D1124FC01E25E41
:102E2000FD4F20812E7F2083875E9D4F0E94020DE3
:102E3000C9C781E080930001C7CF8091000188233A
:102E400009F4A2C6480120EE821A91084090E701D9
:102E500080918701482A80916A03482A38E08316C6
:102E6000910408F086C098012770332781E090E034
:102E700001C0880F2A95EAF7552009F477C0482A3F
:102E8000D7018D919C910E94A00821E030E0F901CA
:102E900002C0EE0FFF1F8A95E2F7FF83EE832090BA
:102EA0006C0430906D0460908401709085011D82E7
:102EB0002D81E22FF0E0EE0FFF1FE652FD4FC080A4
:102EC000D180C114D10409F4C3C6411005C0D60194
:102ED00012968C91811187C0F601838190E02E813A
:102EE0003F8182239323892B09F47DC08085982F0D
:102EF000977009F487E038E08316910408F053C016
:102F0000552009F44CC086958170882309F46BC064
:102F1000D601AD90BC900A151B0519F4552009F493
:102F200062C0C214D30409F45EC0D6011D96ED91AF
:102F3000FC91309721F08081882309F454C0642DDE
:102F4000C6010E940D05882309F44DC00A151B0512
:102F500009F089C70115110509F48AC751108AC7FC
:102F6000A614B70409F03FC0512C84C780954822AD
:102F700087CF552009F455C610938501009384012D
:102F80000E946B04609363047093640480936504EF
:102F90009093660410926B0410926A0471CF82FBC6
:102FA000882780F9B2CF5520F1F08170AECF0E9412
:102FB00020127EC70497813A910548F48A2D0E9419
:102FC0005D08552009F4E0C50E94910CFDCE0E94D9
:102FD000910C8FE19EE40197F1F700C000008A2D6B
:102FE0000E94EF12EECF9D819F5F9D8361CFFC0118
:102FF000208131810217130709F0BFC55110BFC5E9
:103000001092690480E00E947112BEC5902F812F3A
:1030100003C6F901858181FF2FC6C9010E94E80C12
:103020002BC68091110181608093110153C680915C
:1030300011018E7F809311010E942A0D4BC6809151
:1030400011018F7E013E110531F0053E1105C9F4D5
:10305000809111018F7D809311018091110180FF7A
:1030600048C6D70112968C910832110528F50E3109
:10307000110508F072C00430110580F5811135C6C4
:1030800038C6C8019056811540E2940720F0905E42
:103090008115904110F78091110182FF2AC680911D
:1030A000A80381FD26C625EF31E040E0B60190E09F
:1030B00080E00E94CF141DC60933110558F40D326B
:1030C000110518F40B321105C9F69091A60392FD73
:1030D000D5CF08C004361105C1F3D0CF9091A60317
:1030E00094FDCCCF882309F4A8C08091E70190918A
:1030F0006A03892B8D7FB1F11092B2031092B10354
:103100008091A60381FD2EC0F80143E0F695E79576
:103110004A95E1F7EE71FF27E559FC4F98012F70B2
:10312000332781E090E002C0880F991F2A95E2F7CB
:103130008095909520813181822393239183808390
:1031400060E0C8010E94BA148091E7018D7F0E945F
:10315000070882E00E94740D37CE9091A60393FD7C
:103160008DCFC0CF88E0F701A5EFB1E001900D92BF
:103170008A95E1F71092F7011092F9011092F80187
:103180008091B1039091B20308171907D1F52091EE
:10319000A60325FF36C03091110131FF02C026FF82
:1031A00030C02091AF033091B0035601A21AB30A88
:1031B000B7010E94A30BA816B90618F580916A03FF
:1031C00081FF08C08091110180618093110182E02C
:1031D0000E94220880916A0385FF08C08091110136
:1031E00080628093110180E20E94220860911101A7
:1031F000669561708091B1039091B2030E94BA14F8
:10320000E3CD8091E70190916A03982B2091110101
:1032100091FB21F9209311018D7F0E9407081093E3
:10322000B2030093B103D092B003C092AF03809178
:1032300011018460809311018CCF970140E0B601A9
:10324000C8010E94CF14C0CD053F4CE5140709F416
:1032500063C008F45BC0063F8CE5180709F462C040
:10326000D70112963C91332309F4CCC51092700417
:103270000330BDE51B0708F061C00A3FECE51E07FF
:1032800030F4C80182509C45449708F063C00E9406
:10329000D60A909369038093680302315CE51507B1
:1032A00009F49EC108F0EEC009309CE5190709F445
:1032B00075C108F0B8C00530BCE51B0709F462C150
:1032C00008F09FC00330FCE51F0709F453C108F064
:1032D00055C180916803816002303CE5130709F411
:1032E000CEC080916803909169030E94810B0E9477
:1032F000CD0D6ACD07E225EE45EE68ED7CE514C5FF
:1033000006E221EE40EE63EF7CE50EC507E225EE16
:1033100044EE64EF7CE508C506E221EE42EE65EF7F
:103320007CE502C507E225EE46EE66EF7CE5FCC4CF
:1033300008E221E045EE69ED7CE5F6C4053AFDE5DD
:103340001F0709F4A4CF08F055C001364DE5140756
:1033500009F49DCF06318CE5180709F458C50A35E4
:103360005DE5150709F495C108F06EC101159CE5EE
:10337000190709F474C10E3D1C4509F47DC1F7011C
:1033800086819781009709F488C10E947B06182FD7
:10339000092FF701C280D580D2943FE0D3228091DB
:1033A000DC018770C1F0AC2CCC20B1F0892F807F7C
:1033B000803421F080E2810F883068F080916903C9
:1033C00082FF09C082E00E94740D8091DC01877049
:1033D000AA24A3948111A12C902E92942FE09222E2
:1033E000FBE0F91508F4E6C1E92DF0E0EE5EFF4CD4
:1033F0000C942E2FC8018D5A9D45039708F0AACF33
:1034000046CF80916803806207304CE51407B9F11C
:1034100080916803806108305CE5150780F1809138
:10342000680380642CC00D308CE5180709F4C0C017
:1034300090F4809168038E7F0B30ACE51A07F9F0A9
:10344000809168038C600C30BCE51B07C0F0809154
:1034500068038D7F14C00F30ECE51E0709F4B8C077
:1034600008F4AAC000312CE5120709F4B5C0809118
:1034700068038F7B01313CE5130709F032CF80935D
:1034800068032FCF0F3F4CE5140709F4B3C0A8F52C
:103490000A3F8CE5180709F479C0C0F40431ACE5A3
:1034A0001A0709F4B5C008F4A1C00531ECE51E0700
:1034B00009F017CF8091680382FB992790F921E0EA
:1034C000922790FB82F990FB83F9D9CF0C3FFCE562
:1034D0001F0709F475C008F45DC00D3F3CE51307F4
:1034E00009F472C08091690383600E3F4CE51407B4
:1034F00009F0F7CE80936903F4CE01365DE5150738
:1035000009F491C090F401309DE5190709F489C0D0
:1035100008F474C060E00230BDE51B0709F0E1CE9D
:103520008EE090E00E94CA2FDCCE0D3AEDE51E073A
:10353000E9F060F490916803892F8E7F90FF81609D
:10354000053A2DE5120709F49ACFCBCE0E3A3DE5A8
:10355000130751F10F3A4DE5140709F0C2CE9091CF
:103560006903892F877F93FF8860C4CF80916903A7
:103570008860C0CF80916803826081CF80916803AA
:1035800084607DCF80916803886079CF80916903E2
:103590008160B0CF809169038260ACCF0E94CD0D75
:1035A0008091680380686BCF80916903877FA2CF89
:1035B000809168038B7F63CF80916803877F5FCFA3
:1035C000809169038E7F96CF809169038D7F92CF22
:1035D000809168038F7E53CF809168038F7D4FCF9A
:1035E0000E94CD0D809168038F7749CF8091680349
:1035F000837F45CF809169038C7F7CCF8091690365
:10360000982F909591708E7F892B90FB81F972CFC6
:103610000E94CD0D90916803892F97FB87F9805800
:103620002ECF61E07DCF90916803892F8F7E94FF2C
:10363000806125CF80918601811104C089E20E94BA
:103640005008C2CC85E3FBCF0C35BDE51B07B9F0B4
:1036500010F1073A1D4509F092CE0E94EB110E942D
:10366000CD0D2FE73AE146E0215030404040E1F7F0
:1036700000C000000E944B040E948715EECF80918D
:10368000690382FB882780F991E089270E94900DC9
:1036900076CE81E0FBCF80E0F9CF8281008111817D
:1036A000882369F0C8010E94330AD82E682FC80108
:1036B0000E94D408B8018D2D0E94160A66CEC8015A
:1036C0000E94A008D82EF6CF202F2F70B22E802F68
:1036D000807F19F0B29490EFB922CC20A9F0BB20E2
:1036E00059F080E2810F883010F0111107C08B2D46
:1036F0000E9429080E94910C812F5AC08091980441
:10370000B82AB0929804F6CF812F0E942012BB20D5
:1037100009F450C080E2810F883010F0111104C00C
:103720008B2D0E94220803C08B2D0E941B080E9433
:10373000910C40C0302F3F70B32E802F807F80329D
:1037400019F0B29480EFB822112321F1113009F45D
:10375000AEC0CC2009F4B7C0DD2009F47FC020E062
:10376000D7014C9111965C91119712966C9112971A
:1037700013967C91139714968C910E948C0A8091D9
:10378000A80381FDB9CFF701858180FFB5CF8F7088
:10379000858364C08091690382FD40C0CC20C1F163
:1037A000BB2029F08B2D0E9429080E94910C80E0FB
:1037B0000E94EF12A92DA850BB0B149710F40E9481
:1037C000AF04812F902F0E940A098111B7C1109276
:1037D000890110928801AA20B1F08091DC0180FD5E
:1037E00012C0D70112961C928595859585950E94E9
:1037F000A50DC7010E94F2158091DC018595859584
:1038000085950E94670D60E0C7010E94AF0AECCA6F
:1038100080E00E942012BB2069F282CFCC2011F1FF
:10382000D11004C08091E7018B2919C041E0D41266
:1038300006C08091E7018B290E940708BBCF8091C9
:10384000A703823078F3D812EDCF0E94FC07909145
:1038500087018B2D892B8913809387018B2D0E94E3
:103860001912A8CFD11003C00E94FC0717C0809185
:10387000A70351E0D51216C0823008F49BCF809187
:103880006A038B2109F496CF0E94FC07909187016F
:103890008B2D809589238913809387018B2D0E941E
:1038A000121288CF823000F3D812DECF83CF8091FE
:1038B000AD03CC2021F08D1508F47CCFCFCFD816E6
:1038C00008F078CFEBCFDD2049F38091AB039091E6
:1038D000AC03193321F08091A9039091AA030E94AF
:1038E000B709812F0E94201265CF802F869586957B
:1038F000837069F0813009F05DCF812F902F937034
:10390000C11002C090E080E00E94830453CF812F59
:10391000902F9370C11002C090E080E00E94990443
:1039200049CF802F837091F5C11044CF412F42952C
:1039300046954770440F440F812F8F70042E01C0AD
:10394000880F0A94EAF7212F207114FF07C02FE097
:1039500030E001C0220F4A95EAF72095302F3695C6
:1039600036953370323069F050F44091E8013130CF
:1039700029F0822B84230E94C80D1CCF842B822B1C
:10398000FACF282B8091E8018227F5CF8695CC20AD
:1039900011F0802F8170882309F40CCF412F4295BC
:1039A00046954770440F440F812F8F70042E01C03D
:1039B000880F0A94EAF7212F207114FF07C02FE027
:1039C00030E001C0220F4A95EAF72095302F369556
:1039D00036953370323069F050F4409197043130AD
:1039E00029F0822B84230E94560DE4CE842B822B57
:1039F000FACF282B809197048227F5CFF02FFF7004
:103A0000BF2ECC2029F08F2F0E94A50D812F27CF0C
:103A1000812F0E9412128B2D0E94670DCBCE123F78
:103A200089F160F4103FB9F0113F81F0CC2009F426
:103A300080C0D11061CE802F8F7128C0133F49F113
:103A4000143FA1F78091690382FD2FC0802F8F71F1
:103A5000CC2011F31BC08091AD03CC2079F0D81697
:103A600008F0A8CE202F2F7181E090E001C0880FD0
:103A70002A95EAF7909197048927B5CF8D1508F418
:103A800099CEF0CF802F8F71C110C6CF0E94A50DA7
:103A900091CE80E0CC2009F4A6CF81E0902F9F71D9
:103AA00001C0880F9A95EAF79ECF8091A7038230D4
:103AB00040F1CC20D1F09091DC019770943041F42A
:103AC0000E942F08802F8F710E94670DA12C72CE4B
:103AD000D816E0F7202F2F71B22E822F0E94A50D4D
:103AE00063E08B2D0E94B10DF1CFD81630F00E940B
:103AF0002F0864E0802F8F71F5CF81E00E94740D54
:103B0000E5CFCC2059F0302F3F71B32E832F0E9488
:103B1000A50D63E08B2D0E94B10D4CCE81E00E947B
:103B2000740D41E04D1508F045CE82E00E94740D01
:103B300041CED110CACE802F8F716ECFCC2019F01C
:103B4000D11045CE48CED11042CE20E0F7014081C1
:103B500051816281738184810E948C0A8091A803C3
:103B600083FF35CE8091880190918901029709F0F9
:103B70002ECE812F0E9479132ACE552029F0DC0108
:103B800018968C9185FF3ECAC80197558F3F9105C5
:103B900011F008F071C05801BB24BEE00B9FF0018A
:103BA00011249F01275E3D4F6901D70112968C9128
:103BB000E25EFD4F908180FB90F99083882309F4A9
:103BC00028CA0E9477049093F4018093F301F601D0
:103BD00082818F5F82838091980490916A03892B00
:103BE00083838091E70184830680F781E02D3097FD
:103BF00031F0D6011C966D917C91C60109958EE03D
:103C00008A9DF0018B9DF00D1124E75EFD4F8581AB
:103C100081FFFCC990E080E090937104809372046E
:103C20002BC080918401909185010817190781F4B8
:103C30001092850110928401109263041092640422
:103C4000109265041092660410926B0410926A043C
:103C500080916C0490916D04009709F495CFA8E0D1
:103C60008A16910408F0C3C9642D0E940D058111C4
:103C700003C081E00E9471128091A60380FF39C0C9
:103C80000E9477046C01D70112968C91882309F465
:103C9000D6C98091110182FF08C025EF31E040E0D4
:103CA000B60190E080E00E94CF140B31BCE51B0709
:103CB00009F4B7C90C31ECE51E0709F4B8C99091B5
:103CC0001101892F8E7F90FF81600A31FCE51F076B
:103CD00009F4B0C9C8019056811520E2920728F076
:103CE000905E8115904108F0B8C91092B20310920D
:103CF000B103033FBCE51B0709F402CB08F0A4CADB
:103D0000083DFCE51F0709F4F5CA093D2CE512073B
:103D100009F40ECB073D3CE5130709F0A1CA06E202
:103D200021EE41EE67ED7CE5C7010E943C144CC8D2
:103D30000031FFE51F0709F442C801312FE51207E2
:103D400009F040C082E03CC800313FE5130709F4A8
:103D50004FC801314FE5140709F44EC86801E7E583
:103D6000DE1AFFEFCF16D10409F060F56FE072E0C4
:103D70008C2D0E948F0B892B29F58EE08C9DF001F4
:103D80008D9DF00D1124E75EFD4F8281813009F099
:103D900035C880910F0290911002892B99F0809183
:103DA000110290911202892B69F080911302909177
:103DB00014022091150230911602822B932B892B2D
:103DC00009F426C8D70112965C90552009F435C82D
:103DD0000F35BDE51B0709F42CC80036EDE51E07BD
:103DE00051F00E35FDE51F0709F027C8809100014D
:103DF000882309F41EC81092000180E00E9471120D
:103E00000C94E41606315CE5150709F0B8CA8091F8
:103E10006A03982F9A7A2091A50320FF04C0482FA7
:103E2000447409F090E021FF04C0482F417109F06B
:103E300090E022FF04C0482F487809F090E023FF6B
:103E400003C0827209F090E0332309F4F3CB81E0E0
:103E5000911101C080E08093860189E2911185E390
:103E60000E945D08B1C8A114B10409F079C8512CB1
:103E7000B12CA12C80E00E947112D0926D04C092EE
:103E80006C0481E080936904F60185818093670466
:103E900051100EC0AB2861F0F601808191819C0128
:103EA00024503109213A310508F081C80E94500898
:103EB000D6011696AD90BC90C5019A9581159F418B
:103EC00010F4E0EEBE2277247394C5010197803B85
:103ED0009D4508F0712CD6011996ED91FC911A9729
:103EE000309731F01B966D917C9181E00995782295
:103EF000772079F0F601868197810E9425098093C9
:103F00006804C501F8E08F16910408F053C80E94B8
:103F1000BC040E94910C55C8B0E0A0E0E2E9FFE1CA
:103F20000C94452F80919501807F31F4809192010E
:103F3000C091D901811107C0CDB7DEB7E8E00C947C
:103F4000612F2196C770809198018C17A9F3F0908A
:103F50009001E0909101C0909301D0909401A6014E
:103F60006E2D8F2D0E942D05D0E08111EACF8E019C
:103F700083E0000F111F8A95E1F7F801E756FE4F25
:103F800081818E11DECF80818F11DBCF8281811103
:103F9000D8CFE380F480EC18FD0860E080E991E080
:103FA0000E94AF0A60E971E00E94A30BE816F906CF
:103FB00040F6809195018F70806180939501F801A2
:103FC000E256FE4F80818F708061808380E991E0AE
:103FD0000E94F2150E949608AFCFA5E1B0E0E3EF92
:103FE000FFE10C943E2F8C0185E0F801DE01519633
:103FF00001900D928A95E1F7D8015C9011966C9032
:1040000011971296EC9012971396CD90DC9060E089
:1040100080E991E00E94AF0A80E9A82E81E0B82EE5
:104020008090930190909401A401609191018091FE
:1040300090010E942D058111A8C1F0909201F60116
:10404000E819F9094F0160E0FF2009F44BC1C501EF
:104050000E94AF0AB5010E94A30B709095018816CB
:10406000990608F0F2C04091930150919401B090EC
:104070009001A0909101872D807F6A2D09F08CC05E
:104080008B2D0E942D05FE2C811127C0D801119681
:104090008C9111978A1121C08C918B111EC0209197
:1040A00096013091970116968D919C9128173907AA
:1040B000A1F4E11012C0872D8F708061809395016B
:1040C00080E991E00E94F21580919501F8018583C5
:1040D0008F2D6596EFE00C945A2FA601662D852D45
:1040E0000E942D05D82E81E08E25D11080E080FF22
:1040F00018C04E2D662D852D0E947608882389F0E4
:104100008091A80380FF0DC080E991E00E94F21524
:1041100088E0E0E9F1E0DF011D928A95E9F7F12CF2
:10412000D7CF81E08E25D11080E0B82FB170CB2E93
:1041300080FF29C04E2D662D852D0E947608D82E31
:10414000811121C0598A6A8A89899A890E94620AE2
:10415000292F22952F70223050F0243078F49F7050
:1041600051F0F8019581907F31F4FD2CB1CF9F7013
:1041700011F08823D1F3805E8830B8F3C8010E9423
:10418000F215DC2CF2CFEE2009F4A2CF809195013C
:10419000816080939501C3CF8B2D0E942D058111E5
:1041A00024C0D80111968C9111978A111EC08C9150
:1041B0008B111BC0209196013091970116968D911D
:1041C0009C9117972817390781F4E1100EC01596B6
:1041D0007C92C8010E94F21588E0F801A0E9B1E0E4
:1041E00001900D928A95E1F773CFC8010E946F0A82
:1041F000882339F1EE2029F1809195018032A0F0D9
:1042000020919001309191013A8729871B86DD86A4
:10421000CC868E878091960190919701988B8F879D
:10422000CE0109960E94F21588E0F801A0E9B1E0FC
:1042300001900D928A95E1F70E948C1FFF24F39460
:1042400047CFC8010E94F215F9CF872D807F09F46E
:104250005BCF90909001809091014091930150919B
:104260009401682D892D0E942D0581111CC0F80133
:104270008181881118C08081891115C02091960113
:1042800030919701868197812817390761F4E110F1
:104290000AC07582C8010E94F21588E0D5011D92FE
:1042A0008A95E9F715CFC8010E946F0A882349F261
:1042B000EE2039F280919501803208F4B5CF20913B
:1042C0009001309191013A8329831B82DD82CC8257
:1042D0008E83809196019091970198878F83CE016C
:1042E0000196A0CF80E991E00E94AF0A60E971E0F9
:1042F0000E94A30B8816990680F6FE2CEE2009F486
:10430000A0CFE0909001D090910140919301509105
:1043100094016D2D8E2D0E942D05811128C0F8016C
:1043200081818D1124C080818E1121C02091960140
:10433000309197018681978128173907C1F48091C0
:10434000A80382FD49CF9091950190FD45CF907FC4
:1043500009F442CF809195018583903F09F439CFCC
:10436000982F907F905F8F70892B858332CFC80103
:104370000E946F0A811158CF8091950181608093CE
:104380009501C8010E94F215A3CEEE2009F459CF81
:10439000C8010E946F0AF82E882309F452CF88E0E2
:1043A000F801A0E9B1E001900D928A95E1F78091C2
:1043B0009001909191010E94620A0E948C1F88CE08
:1043C000A0E1B0E0E6EEF1E20C944B2F29873A87AA
:1043D0004B875C876D877E878F87988BCE01099688
:1043E0000E94ED1F81112FC088E0FE013996DE0189
:1043F000119601900D928A95E1F74C855D856A854D
:1044000089850E942D0581111EC0A0919801B0E000
:10441000CD010196877099272091D9012817190697
:10442000E1F093E0AA0FBB1F9A95E1F7A756BE4FA4
:1044300098E0FE01319601900D929A95E1F78093F4
:1044400098010E9496088091D90190919801891352
:1044500012C06096E2E00C94672F0E94CD0D10927E
:1044600098011092D90188E0E0E9F1E0DF011D92A6
:104470008A95E9F7E8CFB8E08B9FC00111248756F1
:104480009E4F0E94ED1F882321F38091D90190E077
:104490000196877099278093D901D5CFEF92FF922B
:1044A0000F931F93CF93DF938091B603882361F01E
:1044B000C091B5038CE0F82E8091B603C81748F080
:1044C0001092B6031092B503CDB7DEB7E6E00C94B8
:1044D000632FEE24E394EC0EE092B5030C2F10E072
:1044E000CF9DE0011124C954DC4F4B815C8169816F
:1044F00088810E942D0581111DC08E819F81892B8D
:1045000021F488859985019651F4288139814A8161
:104510005B816C817D818E819F810E94E021F09E74
:10452000F001F19EF00D1124E954FC4F1482138226
:1045300010929804CE2DC0CF10925A0410925904B4
:104540001092120180915804809357040E946605CE
:104550000E944E220895B0E0A0E0E1EBF2E20C945C
:104560003C2FC091570497E0892E01E010E02CE029
:10457000322E3EEF932E44244394809158048C13A2
:1045800009C00E944E220E946605CDB7DEB7E1E168
:104590000C94582FD0E0FE01EE0FFF1FE15BFB4FA4
:1045A00080819181889ED001899EB00D1124A95EE1
:1045B000BB4F14962C911497211158C05090B603FC
:1045C000E7EBF3E030E020E0712C5D01251508F009
:1045D0004BC0E284F384D501CD90DC906FEF7FEF88
:1045E000612C462D50E0DA01AA0FBB1FAC0DBD1D9A
:1045F0000D90BC91A02D109731F0EA16FB0609F43E
:10460000BA016394EECF6F3F7607A9F1D80102C0DB
:10461000AA0FBB1F6A95E2F77A2AB801062C02C0DE
:10462000660F771F0A94E2F7AB01415051097416E7
:104630001506F9F4329EF001339EF00D1124E95471
:10464000FC4F889ED001899EB00D1124A95EBB4FFE
:1046500012962D913C9113973783268390829182F5
:104660009187808715964C920E9438052196C370D9
:1046700084CF148213822F5F3F4F3C96A7CFA9E1CE
:10468000B0E0E5E4F3E20C943B2F942F498B252F07
:104690005A8B6B8B7C8B8D8B4C895D89622F892F1C
:1046A0000E942D05811109C0809188019091890196
:1046B000019690938901809388018B8981111092D2
:1046C00098041D861E861F86188A85E0FE01719655
:1046D000DE01199601900D928A95E1F780916903A8
:1046E00082FF1EC080918D0390918E03892BC1F0B3
:1046F0000E9477042091DA013091DB01821B930B39
:1047000020918D0330918E038217930720F08091C2
:10471000DC0182FFE2C10E94360881110E94FC0781
:104720004C855D856A8589850E942D05811111C0A2
:1047300061E0CE0109960E94AF0A6C018B8527EFDC
:10474000C2162CE5D20681F4882321F181E0809302
:10475000120129853A854B855C856D857E858F851F
:1047600098890E94E021C6C038EFC3163CE5D30605
:1047700029F4882379F00E949C22EBCF49EFC416DC
:104780004CE5D40639F4882329F080911201811177
:10479000F2CFDCCF07E114E0512CB12CA12C222464
:1047A0002394312C2EEF422EF80140815181882430
:1047B0008A94982C20E0822F90E0FC01EE0FFF1FDE
:1047C000E40FF51F608171816115710531F0C61626
:1047D000D70609F44C012F5FEECFF12CFFEF8F16B7
:1047E0009F0609F449C0F8014481F09012018F2D11
:1047F000411180E0F82FF170FF2EF801E5808681ED
:104800009B85992309F4F8C0FF2009F4F5C0609056
:10481000A1037090A203E11013C0A101082C01C0F4
:10482000440F0A94EAF7842B86838091B303909116
:10483000B4038615970520F47092B4036092B30315
:10484000C10102C0880F991F2A95E2F70197F8016C
:1048500026812817190681F48091590490915A04F1
:10486000009709F44BC00E945C046816790608F0B2
:1048700045C021E0F80124835F28FFEFAF1ABF0A8B
:10488000095F1F4F28E0A216B10409F08DCF8B8578
:10489000882309F40DC1552009F40AC10E94770448
:1048A00090935A04809359048091B603883010F590
:1048B00091E0980F9093B60398E0FE013996DE01DF
:1048C000119601900D929A95E1F73CE0839FC0010B
:1048D000112489549C4F28E0FE013196DC0101909F
:1048E0000D922A95E1F72FEF3FEFFC0131872087EA
:1048F000D386C2866996E2E10C94572F80915704C3
:1049000050915804982FF0E0E0E0851314C0909384
:104910005704E017F10709F4AFCF90E0FC01EE0F68
:10492000FF1FE15BFB4FB182A08201968370992744
:1049300080935804A1CF682E712CF301EE0FFF1F56
:10494000E15BFB4F2081318147E0429FD001439FD3
:10495000B00D1124A95EBB4F6D917C911197798F99
:10496000688F40E020E030E0E32FF0E0EE0FFF1F23
:10497000688D798DE60FF71F8080918081149104F6
:10498000E1F0F8010190F081E02DFF8BEE8B20E04B
:1049900005C08616970609F44F2D2F5FE22FF0E031
:1049A000EE0FFF1F6E897F89E60FF71F608171810F
:1049B0006115710571F73F5FD7CF4423D1F0F8013E
:1049C000231708F0FD0121E024830E171F0721F4AF
:1049D00090935704F42E50CF981305C0AE17BF071D
:1049E00011F49F5F937093012F5F3F4F822F83706D
:1049F0008CCFF0E0E0E0F7CF90E0E11020C0B10113
:104A000002C0660F771F2A95E2F79B0121503109FA
:104A10008217930731F4442309F448C0C5010E946A
:104A20003805C101082C01C0880F0A94EAF7982FB5
:104A30009095F801868189238683FE2C1DCF9C01E9
:104A4000082C02C0359527950A94E2F7A901417018
:104A50005527BC016150710986239723892B11F5D5
:104A6000452B01F1F80182819381892BC1F01B82D2
:104A70001C821D821E8249824A820E9477048160C4
:104A8000582F9D838C83F801828193818F8398872F
:104A900029813A814B816D817E810E94E021F8015C
:104AA0001582BFCFF22FF170EF2EBBCFEF2CB9CF15
:104AB0009091570480915804981731F00E94AB22CE
:104AC000552009F446CE16CF0E944E2210925A0469
:104AD000109259040E946605F3CF82E00E94740D83
:104AE0001ACEA5E0B0E0E7E7F5E20C944B2F9093E7
:104AF000650380936403811520E2920730F40E94DD
:104B0000D7122596E2E00C94672F80EF89838A8381
:104B10001B820E9477048160782F9D838C8349815A
:104B20005A816B818D810E943F23EBCF0F931F939E
:104B3000CF93DF938C01EB016FE072E08C2F0E942A
:104B40008F0B892BA1F48091A9039091AA030E9455
:104B5000B709DD27C95FDD4F8881F801128218820D
:104B60008330F1F048F4813059F0823081F0DF91E8
:104B7000CF911F910F9108958430B9F08530B9F726
:104B800080910F0290911002009789F306C08091E6
:104B9000110290911202009799F30E947125E7CFBC
:104BA0008091130290911402F6CF8091150290919A
:104BB0001602009791F720910F0230911002809118
:104BC00011029091120221153105F1F2009729F797
:104BD000C901E3CFA5E0B0E0E0EFF5E20C944B2F84
:104BE0009093650380936403811520E2920730F46B
:104BF0000E94A2142596E2E00C94672F80EF89832F
:104C00008A8381E08B830E9477048160782F9D8363
:104C10008C8349815A816B818D810E943F23EACF29
:104C2000CF93DF93EC010E94EA258091A903909134
:104C3000AA030E94B709CE010E947125DF91CF918E
:104C400008950F931F93CF93DF938C01862F6FE00E
:104C500072E00E948F0B892BB1F4C0910F02D091AA
:104C60001002209781F0F8018281833051F4CE0147
:104C70000E941026CE010E941026CE010E9410260E
:104C800002C08430D0F7DF91CF911F910F9108952A
:104C90000F931F93CF93DF938C01EB016FE072E0D2
:104CA0008C2F0E948F0B892B09F05CC0FE01FF271F
:104CB000D80112968C911297E95FFD4F8130B9F4BB
:104CC00015969C9192FF02C080830AC090FFFCCF92
:104CD00082E0808380911102909112020097B9F4D2
:104CE00080910F02909110020097E1F110C0823084
:104CF000B9F515968C9182FD28C080FD0BC083E02C
:104D000080838091130290911402009701F10E9418
:104D1000EA2528C084E080838091150290911602D4
:104D20000097A9F780910F02909110020097F9F077
:104D30000E9410268091110290911202009739F77B
:104D400080910F0290911002E2CF85E080838091E4
:104D50000F0290911002009729F00E941026F0CFC8
:104D600086E08083DF91CF911F910F91089580910C
:104D7000110290911202B8CFA7E0B0E0E2ECF6E2A7
:104D80000C94422F1F821E828DE4E82E81E0F82EC3
:104D900010E000E0CC24C394D12C27E5A22E21E022
:104DA000B22EF70181917F018F3F09F445C0F8943D
:104DB000E82FE295EF70F0E021A18F70A60102C00C
:104DC000440F551F8A95E2F7CA01922F982B91A3A1
:104DD00092A18095892382A3789400C0EFE4F1E04A
:104DE000912C31E021912F3F09F465C0A22FA295AB
:104DF000AF70B0E090968C9190E02F7002C09595C6
:104E000087952A95E2F780FD56C0832F982A330FA5
:104E1000AE16BF0639F7F701319780818F3F11F049
:104E20000E94210650E55A95F1F7E6E0F0E0EC0F1C
:104E3000FD1FE00FF11F908201301105C9F542E01E
:104E400050E0BE016A5F7F4F8CEE91E00E948F2F91
:104E5000892B99F18E819F819093ED018093EC01D4
:104E600081E08093EB010E9477049093EA018093A4
:104E7000E9018091E9019091EA010E945C040597A3
:104E800000F142E050E06CEE71E085E092E00E94BB
:104E90008F2F10E0892B49F08091EC019091ED016A
:104EA000909306028093050211E01092EB010AC074
:104EB00001E010E076CF80E0A9CF8091EB01811175
:104EC000D8CF10E08091FD018823A1F08695B9F03C
:104ED00081E089838A831B820E9477048160782F16
:104EE0009D838C831092FD0149815A816B818D8154
:104EF0000E943F23812F2796EBE00C945E2F1982AE
:104F000081E0E8CF1F920F920FB60F9211242F93DA
:104F10003F934F935F936F937F938F939F93AF9341
:104F2000BF93CF93DF93EF93FF93D091E900DF70AE
:104F30008091EC00C82FC17080FDC0E81092E9009C
:104F40008091F000877F8093F00078940E94D90DC3
:104F50001092E9008091F00088608093F000CD2BE2
:104F6000CF70C093E900FF91EF91DF91CF91BF9196
:104F7000AF919F918F917F916F915F914F913F91F1
:104F80002F910F900FBE0F901F9018951F920F92A8
:104F90000FB60F9211242F933F934F935F936F930C
:104FA0007F938F939F93AF93BF93EF93FF938091E2
:104FB000E10082FF09C08091E20082FF05C080917C
:104FC000E1008B7F8093E1008091DA0080FF23C0B5
:104FD0008091D80080FF1FC08091DA008E7F80937F
:104FE000DA008091D90019BC80FF9EC082E089BDA3
:104FF00009B400FEFDCF81E080938D048091800490
:10500000811109C00E94C2020E948D038091E200BA
:1050100084608093E2008091E10080FF17C080915E
:10502000E20080FF13C08091E2008E7F8093E20057
:105030008091E20080618093E2008091D8008062DC
:105040008093D80019BC85E080938D048091E100A5
:1050500084FF2EC08091E20084FF2AC019BC82E048
:1050600089BD89B5982F917080FFFBCF8091D800C2
:105070008F7D8093D8008091E1008F7E8093E10046
:105080008091E2008F7E8093E2008091E200816057
:105090008093E20080918E04882309F44AC084E062
:1050A00080938D040E94CD0D0E94AF0480918D04E9
:1050B0008091E10083FF27C08091E20083FF23C03D
:1050C0008091E100877F8093E10082E080938D04EE
:1050D00010928E048091E1008E7F8093E100809198
:1050E000E2008E7F8093E2008091E20080618093F5
:1050F000E20042E060E080E00E945B038091F0000B
:1051000088608093F000FF91EF91BF91AF919F91E4
:105110008F917F916F915F914F913F912F910F9060
:105120000FBE0F901F90189510928D04109280045E
:1051300072CF8091E30087FD93E090938D04B2CF0E
:1051400078941F921FB61F9211248F939F93AF9351
:10515000BF938091790490917A04A0917B04B091DF
:105160007C040196A11DB11D8093790490937A046B
:10517000A0937B04B0937C04BF91AF919F918F91DA
:105180001F901FBE1F9018951F921FB61F921124CB
:105190008F939F93AF93BF938091790490917A04FA
:1051A000A0917B04B0917C044196A11DB11D809318
:1051B000790490937A04A0937B04B0937C04BF910C
:1051C000AF919F918F911F901FBE1F901895CDB7E3
:1051D000DEB7EE970FB6F894DEBF0FBECDBF85B732
:1051E000806885BF85B7806885BF84B7877F84BFA7
:1051F0000FB6F894A8958091600088618093600054
:10520000109260000FBE80E890E00FB6F894809393
:105210006100909361000FBE8FE196E090937B0157
:1052200080937A010E94FA050E944D0C0E94C10BE6
:105230000E94C1090E94C2020E948D038091E20077
:1052400084608093E200789480918D048823A1F09B
:105250001091E9001F709091EC00892F817090FDF2
:1052600080E8182B1092E9008091E80083FD0E94ED
:10527000D90D1F701093E90082E084BD93E095BDC5
:105280009DE797BD80936E000E94BD0A811102C008
:105290000E94621187EF0E9421060FE411E0F801DD
:1052A00081918F018F3F11F00E942106F1E00735B7
:1052B0001F07A9F710920602109205021092ED0145
:1052C0001092EC0190E080E00E94C42F883E9E4F37
:1052D00021F40E94BD0A811102C00E94871582E05C
:1052E00090E00E94BC2F8093F0010E94D60A909318
:1052F0006903809368030E94BC268FE19EE40197B6
:10530000F1F700C000000E94BC268091050280FFDA
:1053100008C06FEF7FEF90E080E00E94E82F0E94CE
:105320004B0483E090E00E94BC2F0E94C80D81E0F6
:105330008093000256985E9A57985F9AE7ECF0E0E7
:105340003197F1F700C000004091000261E072E087
:10535000FB018E2F861B841708F4FDC081E091E0CD
:105360009093760480937504222423943E01FBE2FB
:105370006F0E711CB4E04B2E512C9E012F5F3F4FDE
:1053800069015E0133E0A30EB11C0E94BC2690911E
:10539000F101809105029813EFC09091F201809184
:1053A00006029813E9C00E9477048C018091EE01F7
:1053B0009091EF0108171907A1F08FEF8BAB8CAB21
:1053C0001DAA0E9477048160782F9FAB8EAB4BA9FA
:1053D0005CA96DA98FA90E943F231093EF01009350
:1053E000EE0180916A0490916B04892B09F43EC010
:1053F00040915F0450916004609161047091620477
:105400002FB7F8948091790490917A04A0917B044D
:10541000B0917C042FBF841B950BA60BB70B40915A
:105420005B0450915C0460915D0470915E0484178C
:105430009507A607B707D0F080916A0490916B0496
:105440000E94A21410926B0410926A0410925F04DE
:1054500010926004109261041092620410925B0436
:1054600010925C0410925D0410925E04009171042D
:10547000109172040115110519F18091F3019091B9
:10548000F4010E945C047C0188E0F30111928A958A
:10549000E9F7B301C8010E94A30B8E159F0580F4A4
:1054A00080917104FEE08F9FC0011124FC01E25E37
:1054B000FD4F208122FD04C0875E9D4F0E94020D9A
:1054C00080911201882301F18091590490915A042E
:1054D0000097D1F00E945C042091B3033091B40393
:1054E0002817390788F49091570480915804981729
:1054F00009F47FC00E94AB221092B4031092B30350
:1055000010925A04109259048091A60380FF1EC085
:105510008091110182FF1AC00E9477042091AF038D
:105520003091B003AC01421B530B20910F0130911D
:1055300010014217530750F025EF31E041E0BC0164
:105540008091B1039091B2030E94CF14912C812CD1
:1055500052E0352ED7C089B186FB882780F929B162
:1055600030E0220F232F221F330B90E0232B09F072
:1055700092E0892B8193EDCEA5E0EA2EA2E0FA2EEF
:1055800001EF11E01DAEF70191907F01F8018191CB
:105590008F01891529F189258EAF812C332433940D
:1055A0008EAD8321A9F088AEFDADF9AF91E0892DD4
:1055B000832109F490E09AAF0E9477048160782FEC
:1055C0009CAF8BAF48AD59AD6AAD8CAD0E943F2307
:1055D0008394330C28E08212E3CFF8013197908254
:1055E0003DAD313019F40E946B04FBCE81E08DAFEC
:1055F000CACF0E944E2210925A04109259040E945F
:10560000660582CF092D10E0E9B1E6FBEE27E0F94F
:1056100089B190E0880F892F881F990B892B09F099
:10562000BCC080E08E2BD801AF5FBD4FEC919E2FA8
:105630009370891709F465C0EE0FEE0FE82BEC9319
:10564000EF70F0E0E55AFE4F980121503E4F79018E
:105650008081F9019081890F808320E0843014F1EA
:10566000F801E250FE4F80818F5F8083F801EE0FDA
:10567000FF1FE95AFE4F808191819A8389832B8293
:105680000E9477048160782F9D838C83F801E3501A
:10569000FE4F21E0208349815A816B818D810E94D8
:1056A0003F2321E0F70180818D3F0CF5F801E250A6
:1056B000FE4F808181508083F801EE0FFF1FE75A73
:1056C000FE4F808191819A8389832B820E94770487
:1056D0008160782F9D838C83F801E350FE4F3082E8
:1056E00049815A816B818D810E943F2321E0F7011E
:1056F0008081082E000C990BB2010E941A2F808322
:10570000822A939480910002981608F47BCF81102E
:105710000E946B040E94AF0490910202891721F04D
:10572000809302020E946B0480918D04843009F002
:105730002CCE83E08093E9008091E80082FF25CEA3
:105740008091E80090E085FF05C00E94E102882377
:1057500031F191E08091E8008B778093E800992304
:1057600009F413CE00916603109167038981011536
:10577000110591F18E3F09F071C08A81833020F0CC
:105780008550833008F06AC0EA81EE3008F066C0C8
:10579000F0E0E25EFF4C0C942E2F82E043CF00E25B
:1057A00010E09E012F5F3F4F79018091E80085FD59
:1057B0000AC08091E8008B778093E8000E94E102A4
:1057C000882399F3C6CF8091F100F70181937F017F
:1057D0000150110951F7BDCF8D3009F49AC0B0F4D2
:1057E000843009F47DC040F4823041F108F069C092
:1057F000813001F18FEFF6C2863009F487C008F4DA
:105800007AC08C30B9F780E18A8328C0813109F4ED
:10581000DBC040F48F3009F4AAC008F47EC00E94B7
:10582000310B1CC0833109F4F9C008F4CFC08E3F9E
:1058300009F7AACF1A8289E08B8310C08A8182304F
:1058400009F4EFC2833081F18130A1F60E946B042C
:105850000E94342F6B837C838D839E8380918D0483
:10586000843009F092CD1091E9001F709091EC0006
:10587000892F817090FD80E8182B82E08093E900E9
:105880008091E80080FF0CC050E040E060E270E0F2
:10589000C6010E9412038091E8008E778093E80091
:1058A0001F701093E90071CD80910D0190910E0150
:1058B000892BA1F2809105028B83809106028C8353
:1058C000CDCF8A81823009F095CF6B817C818D812B
:1058D0009E810E94342F86E290E00E94CA2FBECFA4
:1058E0004C816B818A810E94E60998278927982735
:1058F0009E838D83B3CF2D813E813227232732278C
:105900004C816B818A810E94410BA8CF0E94D610E6
:10591000A5CF82E08A8389E58FCFEC80F12CFDE171
:10592000EF16F10408F09ACF8A809B80982489248E
:1059300098248E010F5F1F4FE00EF11EC4018955A0
:105940009E4FE016F10609F489CF29E5821622E080
:10595000920650F40E94BC2FF8018483FFEF8F1A47
:105960009F0A0F5F1F4FEACFF8011482F7CF809193
:105970000D0190910E01892B09F470CFEC80F12C70
:105980002DE1E216F10408F069CF0A811B8110278E
:1059900001271027CE0101964C01E00EF11EC8012F
:1059A00089559E4FE016F10609F458CF0935E2E01B
:1059B0001E0720F4F40164810E94CA2FFFEF8F1AA2
:1059C0009F0A0F5F1F4FEBCF83E01ECFEC80F12CBF
:1059D0002DE1E216F10408F041CF8A809B809824E3
:1059E000892498248E010F5F1F4FE00EF11EC40121
:1059F0008796E016F10609F431CF30E6831691045C
:105A000050F40E94BC2FF8018483FFEF8F1A9F0A85
:105A10000F5F1F4FECCFF8011482F7CFEC80F12C11
:105A20002DE1E216F10408F019CF0A811B8110273D
:105A3000012710270036110508F010CF80E690E00E
:105A4000801B910B8E159F0508F408CFCE0101969F
:105A50004C01E00EF11EC80187960E151F0509F4D2
:105A6000FDCE0036110520F4F40164810E94CA2F96
:105A7000FFEF8F1A9F0A0F5F1F4FEDCF88E0E4E121
:105A8000F1E0DE01919601900D928A95E1F780E2B6
:105A9000F60111928A95E9F785E0898388E0FE0195
:105AA000B196DE01159601900D928A95E1F7D6CE5A
:105AB00080E989832A821B821C82D0CE8C81682F48
:105AC00070E0762F66278B81860F972F911D092E08
:105AD000000CAA0BBB0B45E0880F991FAA1FBB1F28
:105AE0004A95D1F7AC01BD01405E5F4F6F4F7F4FCC
:105AF000481759076A077B0708F4B0CE8039F1E0F0
:105B00009F07A105B10508F0A9CE413921E0520750
:105B10006105710520F040E951E060E070E0481B4C
:105B2000590BBC01605C7E4FC6010E94862F96CE49
:105B30004EE150E06FEF70E0C5010E94A52F80910B
:105B40000D0189830A838ACE81E090E090936703F8
:105B50008093660382E390E09093040280930302B3
:105B60000E9477047BCE80910D0189830A83809106
:105B7000030262CE0B811C8140E250E06FEF70E0C7
:105B8000C6010E94A52F20E333E0A0ECB3E090E033
:105B900080E0AC014E5F5F4F4132510508F05ECEB0
:105BA000F901659174910617170730F48C0D9D1D4E
:105BB000FC0171836083CA01245F3F4FA217B307C2
:105BC00041F74CCE4B815C8180E393E020EC33E0E5
:105BD000FC01659174914617570709F4F4C00C96BF
:105BE00028173907A9F706CE8B819C8100E313E0C3
:105BF000F801259134918217930709F4F5C0045FE9
:105C00001F4FF3E0003C1F0799F7EE24EA94FE2CA7
:105C100006C10E94A21022CEEB81E73008F01ECE12
:105C2000F0E0E45DFF4C0C942E2F8EE1F501119213
:105C30008A95E9F788E089838A83FECD8C819AE092
:105C4000F92E8E010F5D1F4FF8012F2D11922A950D
:105C5000E9F7B8010E948F0B8983F801DE011296E3
:105C600001900D92FA94E1F7F9CD1C818AE0FE01D2
:105C70003596DE01919601900D928A95E1F789A102
:105C80009AA10E9412069AA389A38BA19CA10E94AB
:105C900012069CA38BA38DA19EA10E9412069EA317
:105CA0008DA38FA198A50E94120698A78FA38FEFAE
:105CB000183068F43AE0139FB001112469547F4F03
:105CC0004AE050E0CE0181960E94EE2F80E0898369
:105CD0000E94FA05C3CD6C812AE0CE018196FC01B9
:105CE000322F11923A95E9F7683008F046C0629F6A
:105CF000B0011124695F7E4F4AE050E00E94AC2F52
:105D000080E089838AE0FE01B196DE011296CBCE57
:105D10001C818AE0FE013596DE01919601900D927C
:105D20008A95E1F789A59AA50E9412069AA789A7E4
:105D30008FEF183068F48AE0189FB0011124695F72
:105D40007E4F4AE050E0CE0181960E94EE2F80E027
:105D500089830E944D0C82CD6C812AE0CE01819610
:105D6000FC01322F11923A95E9F7683030F4629FC6
:105D7000B0011124695A7E4FBFCF8FEFC2CF1C8173
:105D80008AE0FE013596DE01919601900D928A958A
:105D9000E1F78BA19CA10E9412069CA38BA38FEF1D
:105DA000183068F48AE0189FB0011124695A7E4FB8
:105DB0004AE050E0CE0181960E94EE2F80E0898378
:105DC0000E94C10B4BCDFC013696259134912115D3
:105DD000310509F40FCD4FE150E0BE016E5F7F4FFA
:105DE000F901099589833ACDF801389625913491C6
:105DF0002115310509F409CF4CE150E0BE016B5F7C
:105E00007F4FC801F90109957C01892B41F4F80104
:105E10003A9685919491009711F0FC010995E982D9
:105E20001DCD86E290E00E94BC2F1B821C821D8249
:105E30008E8314CD97FB072E16F4009407D077FDC0
:105E400009D00E94722F07FC05D03EF490958195F1
:105E50009F4F0895709561957F4F0895EE0FFF1F36
:105E60000590F491E02D09946927962769277827F2
:105E70008727782708952F923F924F925F926F92D3
:105E80007F928F929F92AF92BF92CF92DF92EF92CA
:105E9000FF920F931F93CF93DF93CDB7DEB7CA1B4B
:105EA000DB0B0FB6F894DEBF0FBECDBF09942A8876
:105EB000398848885F846E847D848C849B84AA841E
:105EC000B984C884DF80EE80FD800C811B81AA81AB
:105ED000B981CE0FD11D0FB6F894DEBF0FBECDBF76
:105EE000ED010895AA1BBB1B51E107C0AA1FBB1FF0
:105EF000A617B70710F0A61BB70B881F991F5A9556
:105F0000A9F780959095BC01CD010895FB01DC01B6
:105F100002C005900D9241505040D8F70895FB0102
:105F2000DC0104C08D910190801921F44150504052
:105F3000C8F7881B990B0895FB01DC0102C0019092
:105F40000D9241505040D8F70895DC0101C06D9387
:105F500041505040E0F70895DC01CB01FC01F99974
:105F6000FECF06C0F2BDE1BDF89A319600B40D92A5
:105F700041505040B8F70895F999FECF92BD81BDC8
:105F8000F89A992780B50895A8E1B0E042E050E082
:105F90000C94AE2F262FF999FECF92BD81BDF89AB1
:105FA000019700B4021639F01FBA20BD0FB6F8945D
:105FB000FA9AF99A0FBE08950396272F0E94CB2FC5
:105FC0000E94CA2F252F0E94CB2F242F0C94CB2F59
:105FD0000196272F0E94CB2F0C94CA2FDC01CB01F6
:105FE00003C02D910E94F92F41505040D0F70895E1
:105FF000262FF999FECF1FBA92BD81BD20BD0FB6E5
:10600000F894FA9AF99A0FBE01960895F894FFCF82
:10601000BA0EE20E9010E20E9010150F360F90108F
:106020003F104C10641B641B9A1B9A1B751CDA1BD7
:10603000DA1BDA1B911CFE1C0F1D0F1D3E2D582D67
:106040005E2D2E2C2E2C982DA42DB32D2E2CBA2D5A
:10605000E22DF42D092E0C2E152E1E2E352E6B2E14
:06606000882EAC2EBF2EBD
:106066000148048A0947048509800946040100AFEE
:10607600000101012B723E47503C867D818283E2FE
:1060860000E900EA00B500B600B700CD008301CCF8
:10609600008A01920194012102230224022502268C
:1060A6000227022A02B300B4006F007000F7FF3621
:1060B60035343130C6F0940001010100FF010001C2
:1060C6000000FFFF0000010001FF00402232000136
:0A60D600DE00AC00D203EB030B0464
:00000001FF
